:100000000C9434000C943E000C943E000C943E0082
:100010000C943E000C943E000C943E000C943E0068
:100020000C943E000C943E000C943E000C943E0058
:100030000C943E000C943E000C943E000C943E0048
:100040000C943E000C943E000C943E000C943E0038
:100050000C943E000C943E000C943E000C943E0028
:100060000C943E000C943E0011241FBECFEFD8E04C
:10007000DEBFCDBF0E9440000C9481000C940000B4
:10008000CF93DF93CDB7DEB784E290E02FEFFC0192
:1000900020838AE290E0FC0110828BE290E0FC0178
:1000A00020818BE290E02C60FC01208385E290E0CF
:1000B000FC01108289E290E0FC018081882F90E0B1
:1000C00084709927009749F485E290E0FC01208133
:1000D00085E290E02062FC01208389E290E0FC014F
:1000E0008081882F90E088709927009719F785E222
:1000F00090E0FC01208185E290E02F7DFC012083CF
:06010000D9CFF894FFCFF7
:00000001FF
